S01900006F70656E626C745F73746D3332663734362E73726563F8
S315080000000000052035070008010700080307000857
S315080000100507000807070008090700080000000090
S315080000200000000000000000000000000B070008A8
S315080000300D070008000000000F0700081107000858
S315080000408507000885070008850700088507000852
S315080000508507000885070008850700088507000842
S315080000608507000885070008850700088507000832
S315080000708507000885070008850700088507000822
S315080000808507000885070008850700088507000812
S315080000908507000885070008850700088507000802
S315080000A085070008850700088507000885070008F2
S315080000B085070008850700088507000885070008E2
S315080000C085070008850700088507000885070008D2
S315080000D085070008850700088507000885070008C2
S315080000E085070008850700088507000885070008B2
S315080000F085070008850700088507000885070008A2
S315080001008507000885070008850700088507000891
S315080001108507000885070008850700088507000881
S315080001208507000885070008850700088507000871
S315080001308507000885070008850700088507000861
S315080001408507000885070008850700088507000851
S315080001508507000885070008850700088507000841
S315080001608507000885070008850700088507000831
S3150800017085070008850700088507000800000000B5
S315080001808507000885070008850700088507000811
S315080001908507000885070008850700088507000801
S315080001A085070008850700088507000885070008F1
S315080001B085070008850700088507000885070008E1
S30D080001C0850700088507000801
S315080001C810B5054C237833B9044B13B10448AFF37B
S315080001D800800123237010BDC40000200000000021
S315080001E86455000808B5034B1BB103490348AFF328
S315080001F8008008BD00000000C800002064550008FB
S3150800020808B504F089FC08BD08B504F093FC08BDD8
S3150800021808B502F0C7F808BD08B5064B1B6913F4FC
S31508000228005F01D0002008BD00F040F8FFF7F0FF96
S315080002380120F8E70008024008B5642000F008F82D
S3150800024808BD08B500F00AF808BD7047704770473A
S31508000258014B1880704700BFE000002008B504F07D
S315080002681DFA0E4B1B6898420FD30D4B1B786BB9BA
S315080002780B4B01221A700B4B80229A6104F00EFA76
S31508000288094B1B881844054B186008BD044B002207
S315080002981A70044B4FF400029A61EFE7E400002055
S315080002A8E200002000040240E0000020024B4FF460
S315080002B800029A61704700BF0004024070B58CB00E
S315080002C800240794089409940A940B94234B1A6BF0
S315080002D842F004021A631A6B02F004020592059AA0
S315080002E81A6B42F080021A631A6B02F080020492B3
S315080002F8049A1A6B42F008021A631A6B02F008028B
S315080003080392039A1A6B42F001021A631A6B02F0F7
S3150800031801020292029A1A6B42F002021A631B6BD6
S3150800032803F002030193019B0D4E4FF40003B361DA
S315080003380CAD4FF4005345F8183D2946094801F015
S3150800034899FF8023069301230793089409940A942E
S315080003582946304601F08EFF0CB070BD00380240C1
S3150800036800040240000802402DE9F04190B000243C
S3150800037809940A940B940C940D940E940F9406946D
S315080003880794274B1A6C42F480221A641A6C02F4F2
S3150800039880220292029A1A6B42F008021A631B6BB1
S315080003A803F008030193019B4FF4807303934FF0FE
S315080003B80208CDF810800327059707260896194DD1
S315080003C803A9284601F056FF4FF400730393CDF8A6
S315080003D81080059706940794089603A9284601F0FD
S315080003E849FF4FF4E13309930A940B940C940C23B0
S315080003F80D930E940F940C4C09A9204602F022FA84
S31508000408636823F490436360A36823F02A03A36010
S31508000418236843F00103236010B0BDE8F08100BFEC
S3150800042800380240000C02400048004008B5364A29
S31508000438136823F00F0343F007031360324B1B6856
S3150800044803F00F03072BF9D1304B1A6842F44042E0
S315080004581A601A6842F480321A6003F5E4331A6897
S3150800046842F480221A601A6842F480321A60284BCD
S315080004781B6813F4003FFAD0254B5A6825491140E2
S31508000488254A0A435A605A6824491140244A0A43A5
S315080004985A601A6842F080721A601D4B1B6813F07E
S315080004A8007FFAD01A4B9A6822F0F0029A609A6886
S315080004B822F4E05242F4A0529A609A6822F4604202
S315080004C842F400429A609A6822F0030242F0020255
S315080004D89A600F4B9B6803F00C03082BF9D1114857
S315080004E802F0DCFF002000F061F9094BD3F89020F0
S315080004F822F00062C3F89020D3F8902022F0300248
S31508000508C3F8902008BD00BF003C024000700040B8
S31508000518003802400080BCFF086C40000080BFF02D
S31508000528086C400900E6DF0C08B500F065F9FFF726
S315080005387DFFFFF7C3FEFFF717FFFFF761FEFFF71B
S3150800054863FEFCE782B00A4B1A6C42F080521A64C2
S315080005581A6C02F080520092009A5A6C42F4804251
S315080005685A645B6C03F480430193019B02B070479D
S315080005780038024000B589B0002303930493059315
S31508000588069307930268144B9A4202D009B05DF89D
S3150800059804FB03F5EA331A6C42F000721A641A6C03
S315080005A802F000720192019A1A6B42F002021A636B
S315080005B81B6B03F002030293029B4FF440730393E9
S315080005C802230493032306930923079303A90348DD
S315080005D800F0D2FDDAE700BF0064004000040240DC
S315080005E810B588B0002303930493059306930793DD
S315080005F80368B3F1A04F01D008B010BD144C236BA3
S3150800060843F001032363236B03F001030093009B64
S315080006184FF4C053039302230493032306930A2330
S31508000628079303A90B4800F0A7FD636B43F0800303
S315080006386363636B03F080030193019B636C43F464
S3150800064880436364636C03F480430293029BD3E795
S31508000658003802400000024008B50368B3F1A04F0D
S3150800066800D008BD054A536B23F0800353634FF443
S31508000678C051034800F06EFEF3E700BF0038024099
S315080006880000024010B5174C4FF40003A361164842
S3150800069801F032FD154801F02FFD204601F02CFD2A
S315080006A8134801F029FD134B1A6C22F480221A64A8
S315080006B81A6B22F008021A631A6B22F004021A63EC
S315080006C81A6B22F002021A631A6B22F001021A63E5
S315080006D81A6C22F080521A645A6C22F480425A64C0
S315080006E810BD00BF00040240000C0240000802408A
S315080006F800000240003802407047FEE7FEE7FEE7C2
S31508000708FEE770477047704708B500F081F808BDDE
S31508000718054BD3F8882042F47002C3F888204FF0B6
S3150800072800629A60704700BF00ED00E0DFF834D039
S31508000738002103E00C4B5B58435004310B480C4B23
S3150800074842189A42F6D30B4A02E0002342F8043BC1
S31508000758094B9A42F9D3FFF7DBFF04F0DBFEFFF7F4
S31508000768E3FE7047000005203C57000800000020FB
S31508000778C4000020C4000020A0100020FEE70000E6
S3150800078810B5094B4FF0FF321A6200241C625A62F0
S315080007985C621A611C615A615C619A619C61FFF727
S315080007A871FF204610BD00BF0038024010B5044648
S315080007B80E4B18784FF47A73B3FBF0F30C4A1068AB
S315080007C8B0FBF3F000F014FB68B90F2C01D901202F
S315080007D80AE0002221464FF0FF3000F0D7FA054B11
S315080007E81C60002000E0012010BD00BF04000020A6
S315080007F8000000200800002008B5032000F0B4FA1D
S315080008080020FFF7D3FFFFF79DFE002008BD000074
S31508000818034A1168034B1B780B441360704700BFE3
S31508000828400E00200400002038B5044603F03EFFB9
S315080008380546B4F1FF3F02D0044B1B781C4403F06D
S3150800084835FF401BA042FAD338BD00BF040000207C
S31508000858002800F0A18038B5044690F82030D3B1B6
S315080008682268136823F00203136003F01FFF054686
S3150800087823685A6812F0020F10D003F017FF401BBE
S315080008880A28F5D9636A43F400336362052384F8B2
S315080008982030012038BDFFF76DFEE1E71A6842F0FF
S315080008A801021A6003F002FF054623685A6812F027
S315080008B8010F0DD103F0FAFE401B0A28F5D9636A21
S315080008C843F400336362052384F820300120E1E706
S315080008D8227E012A3DD01A6822F080021A60637EB9
S315080008E8012B3BD02268136823F040031360A37ECC
S315080008F8012B39D02268136823F020031360E37E9E
S31508000908012B37D02268136843F010031360237F3E
S31508000918012B35D02268136823F008031360637F18
S31508000928012B33D02268136823F004031360A368E5
S31508000938E268134322691343626913436268013AFA
S3150800094821681343CB6100206062012384F82030B4
S31508000958A0E71A6842F080021A60C0E7226813689E
S3150800096843F040031360C2E72268136843F0200384
S315080009781360C4E72268136823F010031360C6E7F8
S315080009882268136843F008031360C8E722681368E7
S3150800099843F004031360CAE70120704790F8203033
S315080009A8013BDBB2012B05D9436A43F48023436232
S315080009B80120704770B4434BD3F8002242F0010275
S315080009C8C3F80022D3F8002222F47C52C3F8002286
S315080009D8D3F80022486A42EA0022C3F800224A6984
S315080009E802F01F02012000FA02F2D3F81C42D04393
S315080009F80440C3F81C42CB69B3B9324BD3F80C424E
S31508000A080440C3F80C42CE688D884C6945EA064509
S31508000A18483443F834508E680C884D6944EA0644CD
S31508000A28483503EBC5035C60CB69012B1DD08B6980
S31508000A38002B32D1234CD4F804320340C4F80432CC
S31508000A480B698BBB1F4BD3F814422040C3F814021A
S31508000A580B6A012B2FD01B4AD2F8003223F0010368
S31508000A68C2F80032002070BC7047164BD3F80C4207
S31508000A781443C3F80C420E688D884C6945EA064546
S31508000A88483443F834508E688C894D6944EA0644DC
S31508000A98483503EBC5035C60C9E70A4CD4F8043249
S31508000AA81343C4F80432CBE70648D0F81432134384
S31508000AB8C0F81432CCE70349D1F81C321A43C1F8F6
S31508000AC81C22C8E70064004038B590F82030DBB22D
S31508000AD8012B05D0436A43F400234362012038BD3D
S31508000AE80446022380F820300268136823F00103BD
S31508000AF8136003F0DBFD054623685B6813F0010FF6
S31508000B080DD003F0D3FD401B0A28F5D9636A43F4D0
S31508000B1800336362052384F820300120DFE70020CC
S31508000B286062DCE770B490F820400568AD68013C5F
S31508000B38E4B2012C06D9436A43F4802343620120B0
S31508000B4870BC704715F0E05F5BD0C5F30165022DF0
S31508000B583ED80124AC401C608B68002B3ED10E6839
S31508000B68CB68046843EA465605F118031B01E650A4
S31508000B7803680C6905F1180603EB06135C600B7D20
S31508000B88012B36D0D17993791B0443EA016351794D
S31508000B9843EA01231479016823432C012144C1F847
S31508000BA88C31D17893781B0443EA0163517843EA78
S31508000BB80123117802680B432244C2F88831026877
S31508000BC818352D01535943F0010353510020B7E74F
S31508000BD8436A43F4000343620120B1E74C6843EAD9
S31508000BE8C403CC680668234305F118042401335165
S31508000BF8BEE7036803EB0613596841F48071596028
S31508000C08C0E7436A43F400134362012098E790F863
S31508000C182030013BDBB2012B01D90020704703685D
S31508000C289B68890631EA030301D001207047002032
S31508000C38704730B490F82040013CE4B2012C06D93C
S31508000C48436A43F480234362012030BC7047002975
S31508000C586FD10468E46814F0030F64D0056801F1DD
S31508000C681B0424012C5904F004049460002C6BD14D
S31508000C78056801F11B0424012C59640D14600568E4
S31508000C8801F11B0424012D5905F00205D5600568F4
S31508000C9825446D6805F00F051561056825446D68D6
S31508000CA8C5F30725956105682C446468240C5461C6
S31508000CB804680A011444D4F8B8411C70046814443A
S31508000CC8D4F8B841C4F307245C7004681444D4F80B
S31508000CD8B841C4F307449C7004681444D4F8B8416E
S31508000CE8240EDC7004681444D4F8BC411C710468EA
S31508000CF81444D4F8BC41C4F307245C71046814444A
S31508000D08D4F8BC41C4F307449C7104682244D2F859
S31508000D18BC21120EDA71F9B90268D36843F02003C8
S31508000D28D360002091E7436A43F400134362012025
S31508000D388BE70468246914F0030F8FD1436A43F4D8
S31508000D4800134362012080E7056801F11B042401AA
S31508000D582C59E408546092E70268136943F02003A3
S31508000D681361002071E700000649CB6823F4E063A5
S31508000D781B041B0C000200F4E0600343024A1A43F2
S31508000D88CA60704700ED00E00000FA0530B4154B5C
S31508000D98DB68C3F30223C3F10704042C28BF042421
S31508000DA81D1D062D14D9033B4FF0FF3505FA04F42B
S31508000DB821EA0401994005FA03F322EA03031943D1
S31508000DC8002807DB0901C9B2074B195430BC70471C
S31508000DD80023E9E700F00F000901C9B2034B1954CB
S31508000DE8F4E700BF00ED00E000E400E014ED00E0E1
S31508000DF80138B0F1807F0AD2064B5860064AF021BE
S31508000E0882F823100020986007221A60704701208C
S31508000E18704700BF10E000E000ED00E010B40A4992
S31508000E280C6924F440740C610C6944F440740C6130
S31508000E380C6944F001040C6102604360BFF34F8FEC
S31508000E485DF8044B704700BF003C0240084B1A691E
S31508000E5822F440721A611A6942F400721A611A6910
S31508000E6842F001021A610160BFF34F8F704700BF55
S31508000E78003C0240084B1A6922F440721A611A6942
S31508000E8842F480721A611A6942F001021A610180F5
S31508000E98BFF34F8F704700BF003C0240074B1A69E3
S31508000EA822F440721A611A691A611A6942F0010233
S31508000EB81A610170BFF34F8F704700BF003C0240AC
S31508000EC81A4BDB6813F0020F04D0194A936943F0EA
S31508000ED820039361154BDB6813F0100F04D0144AEE
S31508000EE8936943F010039361104BDB6813F0200FE6
S31508000EF804D00F4A936943F0080393610B4BDB68E8
S31508000F0813F0400F04D00A4A936943F00403936127
S31508000F18064BDB6813F0800F04D0054A936943F043
S31508000F2802039361014BF222DA607047003C0240E3
S31508000F38440E0020094B1B69002B01DB0020704773
S31508000F48064B074A5A6002F188325A601B69002B19
S31508000F5801DB002070470120704700BF003C0240B3
S31508000F6823016745034A136943F0004313610020C8
S31508000F78704700BF003C024038B50446164B0022AD
S31508000F889A6103F093FB0546144BDB6813F4803F1C
S31508000F980AD0B4F1FF3FF7D0CCB103F087FB401B6A
S31508000FA8A042F1D903200DE00C4BDB6813F0F20FD1
S31508000FB809D10A4BDB6813F0010F0AD0074B012247
S31508000FC8DA60002038BDFFF77BFF0120FAE7032027
S31508000FD8F8E70020F6E700BF440E0020003C024070
S31508000FE8F8B51E4C247D012C35D01F4616460D46ED
S31508000FF804461A4B01221A754CF25030FFF7BCFF0B
S31508001008014698B9032C07D8DFE804F002151A1F19
S31508001018F1B22846FFF742FF4CF25030FFF7ACFF13
S3150800102801460F4A136923F0010313610B4B00228B
S315080010381A750846F8BDB1B22846FFF71BFFEBE755
S3150800104831462846FFF702FFE6E732463B4628467A
S31508001058FFF7E4FEE0E70221EBE700BF440E0020B5
S31508001068003C0240084B1A6922F440721A611A6950
S3150800107842F004021A611A6942EA002040F48030F4
S315080010881861BFF34F8F7047003C024010B449B14E
S31508001098012923D0022902D04FF4407403E04FF403
S315080010A8007400E000240F4B196921F44071196196
S315080010B81A6922431A611A6922F0F8021A611A692A
S315080010C842EAC00040F0020018611A6942F4803208
S315080010D81A61BFF34F8F5DF8044B70474FF480745D
S315080010E8E1E700BF003C0240214B1B7D012B3CD0A9
S315080010F870B50E4604461E4B01221A754CF250303E
S31508001108FFF73AFF024658BB4FF0FF3333602368B0
S31508001118012B16D06568A36861680B44AB421FD9D2
S31508001128217B2846FFF7B2FF4CF25030FFF724FF21
S31508001138104A136923F07A031361024678B9013510
S31508001148E9E7207BFFF78EFF4CF25030FFF714FFD4
S31508001158024608490B6923F004030B6100E0356071
S31508001168034B00211975104670BD022210467047B8
S31508001178440E0020003C024000230F2B00F2E180B9
S31508001188F0B583B039E0092200E00022B2403A43BC
S3150800119802346C4E46F824206B4A1468EA4302EA7D
S315080011A804064F6817F4803F01D045EA0406664CE2
S315080011B82660646802EA04064F6817F4003F01D0FF
S315080011C845EA0406604C6660A46802EA04064F68A5
S315080011D817F4801F01D045EA04065B4CA660E4684C
S315080011E822404E6816F4001F01D045EA0402564C00
S315080011F8E26001330F2B00F2A28001229A400C68A4
S3150800120804EA0205AA42F4D14C68661E112C18BFD6
S31508001218012E01D9122C12D186685F000324BC401E
S3150800122826EA0406CC68BC4034438460466826EA45
S3150800123802064C68C4F300129A4032434260C268F8
S315080012485F000326BE40F64332408C68BC40144310
S31508001258C4604A68122A18BF022A13D1DC0808345F
S3150800126850F824E003F007024FEA820C0F2202FA2C
S315080012780CF22EEA020E0A6902FA0CF242EA0E0289
S3150800128840F82420026816404A6802F00302BA4069
S31508001298324302604A6812F0805FAAD02B4A546C1F
S315080012A844F480445464526C02F480420192019AD0
S315080012B89C08A61C234A52F8267003F003029600D7
S315080012C80F22B24027EA0207214A90423FF45DAF4F
S315080012D802F58062904222D002F58062904220D0C0
S315080012E802F5806290421ED002F5806290421CD0B8
S315080012F802F5806290421AD002F58062904218D0B0
S3150800130802F58062904216D002F58062904214D0A7
S3150800131802F5806290423FF436AF0A2236E7012288
S3150800132834E7022232E7032230E704222EE70522B1
S315080013382CE706222AE7072228E7082226E703B029
S31508001348F0BD704700380140003C014000380240B3
S315080013580000024000230F2B00F29480F0B529E024
S31508001368092700E0002707FA05F5B54271D0056890
S315080013785E000324B440E44325400560DD080835CB
S3150800138850F8256003F007074FEA870C0F2707FA76
S315080013980CF726EA070640F82560C5682540C560A3
S315080013A8456825EA0202426082681440846001336F
S315080013B80F2B66D801229A4002EA0104A242F6D106
S315080013C84FEA930E0EF102062F4D55F8266003F0E4
S315080013D80305AD004FF00F0C0CFA05FC0CEA0606DF
S315080013E82A4FB842BED007F58067B84221D007F51C
S315080013F88067B8421FD007F58067B8421DD007F541
S315080014088067B8421BD007F58067B84219D007F538
S315080014188067B84217D007F58067B84215D007F530
S315080014288067B84213D007F58067B84298D00A276C
S3150800143899E7012797E7022795E7032793E70427FC
S3150800144891E705278FE706278DE707278BE70827FC
S3150800145889E70F4D2E68E44326402E606E682640BD
S315080014686E60AE682640AE60EE683440EC60064EA4
S315080014780EF1020456F8245025EA0C0546F82450BD
S3150800148875E7F0BD704700BF00380140000002400C
S31508001498003C01402DE9F04782B00768CA00521A95
S315080014A8930003445A6D1B6D9A4257D8B8469B1A3F
S315080014B8C1EBC104A2000244526C9A4200D31A46F0
S315080014C80C46064602F1030A4FEA9A0A16E009F19B
S315080014D8030A4FEA9A0AE3001B1B9D003544A96CC8
S315080014E8337C00931FFA89F3E2B2384601F086FD89
S315080014F8AB6C4B44AB646B6D4B446B6508EB4413A0
S3150800150803F510639B699BB2534513D3E3001B1B72
S315080015189A003244516D136D99420BD253B15B1A36
S31508001528C4EBC4018A003244D2F844909945CED314
S315080015389946CCE7E3001B1B98000644326D736D89
S315080015489A420FD804F00F040121A140D7F834486D
S3150800155824EA0104C7F83448002000E0012002B054
S31508001568BDE8F0870020FAE7F0B58BB0002800F050
S3150800157891800446056890F8BD3323B3032384F89D
S31508001588BD33EB6B13F4807F01D1002323612068F8
S3150800159801F0C4FA254655F8107B6E460FCD0FC6DE
S315080015A80FCD0FC695E8030086E80300231D0ECB6A
S315080015B8384601F0F9F958B1022384F8BD330125F4
S315080015C828460BB0F0BD80F8BC33FFF709F8D5E715
S315080015D80021206801F0A8FA002315E0D900C81AE6
S315080015E882002244012082F83D0082F83C30A2F8A5
S315080015F84230002082F83F0050649064CA1A91006D
S31508001608214408650133DBB26568AB42E6D300239B
S3150800161815E0D800C11A8A002244002182F8FD1173
S3150800162882F8FC3182F8FF11C2F80412C2F80812CF
S31508001638C21A90002044C0F810120133DBB29D424A
S31508001648E7D8254655F8107B6E460FCD0FC60FCD41
S315080016580FC695E8030086E80300231D0ECB384617
S3150800166801F0A8FA054660B9002384F83830012342
S3150800167884F8BD33636A012B08D0206801F08DFE13
S315080016889EE7022384F8BD33012599E7204600F032
S3150800169817FDF2E7012593E790F8BC33012B0ED026
S315080016A810B50446012380F8BC33006801F069FECA
S315080016B8206801F02DFA002084F8BC0310BD02202A
S315080016C8704738B590F8BC33012B18D00446012367
S315080016D880F8BC33006801F021FA206801F01DFE85
S315080016E8054628B1002384F8BC330125284638BDA9
S315080016F8206801F052FE002384F8BC33F6E7022579
S31508001708F4E768B110B50446032380F8BD33FFF73C
S31508001718D8FF2046FEF7A0FF002084F8BD0310BDB9
S315080017280120704770B504460D460068066C00EB44
S31508001738411303F530639A682169012911D037499D
S315080017488E4254D03DB9C5EBC50293002344D3F85D
S315080017581032002B5CD0E9B2204603F0ABFD00201E
S3150800176870BD12F0080F09D02D498E42F7D912F428
S31508001778004FF4D04FF400429A60F0E712F0200FB9
S3150800178828D112F0280FEAD125498E4202D912F437
S31508001798004F22D1E900491B8A002244D2F80412D4
S315080017A81B69C3F31203C91AC2F81412D2F8041231
S315080017B8D2F808320B44C2F8083235B9C5EBC50267
S315080017C893002344D3F810325BB1E9B2204603F0FC
S315080017D871FDC4E720229A60C1E74FF400429A6077
S315080017E8BDE704F57172012101F028FEEDE712F450
S315080017F8004F09D112F0200F01D020229A60E9B2D1
S31508001808204603F057FDAAE74FF400429A60A6E778
S3150800181804F57172002101F011FE9CE70A31544F54
S315080018280A30544F38B5044603681D6C03EB41115A
S31508001838D1F8082B0E4B9D4207D901F5306112F4F1
S31508001848004F02D04FF400438B60204603F02AFD70
S31508001858074B9D4202D92369012B01D0002038BDC8
S3150800186804F571720121206801F0E8FDF6E700BF6A
S315080018780A30544F2DE9F84F04460568284601F002
S31508001888C9FD08B1BDE8F88F2F460646206801F05D
S3150800189890FD0028F6D0206801F08BFD10F0020FA5
S315080018A804D02268536903F002035361206801F0E3
S315080018B880FD10F0100F15D02268936923F01003E5
S315080018C89361D5F8208008F00F09C8F34343022B23
S315080018D800F08580062B00F0A5802268936943F0FE
S315080018E810039361206801F064FD10F4002F40F09E
S315080018F8AD80206801F05DFD10F4802F40F0F1807E
S31508001908206801F056FD0028C0F25F81206801F0C2
S3150800191850FD10F4006F0AD0D5F8083813F0010FF7
S3150800192840F06D812268536903F4006353612068A7
S3150800193801F03FFD10F0006F15D02268536903F0D7
S315080019480063536194F8F433002B40F05C8101215D
S3150800195884F8F41323685B6DC3F38303C4F8F83378
S31508001968204600F0C1FB206801F023FD10F4805FD3
S3150800197840F04D81206801F01CFD10F4005F40F02E
S31508001988AB81206801F015FD10F0080F40F0BC8106
S31508001998206801F00EFD10F4801F40F0BE81206813
S315080019A801F007FD10F4001F40F0C181206801F01E
S315080019B800FD10F0804F40F0C481206801F0F9FC62
S315080019C810F0040F3FF45EAF23685D6815F0040F46
S315080019D840F0C081226853682B43536052E747F6A4
S315080019E8F07318EA030F3FF478AF4FEAC90BABEB6D
S315080019F809034FEA830AA2444FEA1818C8F30A02E9
S31508001A08DAF80812284601F019FCC8F30A08DAF8C1
S31508001A1808324344CAF80832DAF814324344CAF892
S31508001A2814325AE7082204F57171284601F006FCB3
S31508001A38C8F30A184FEAC903A3EB09018A00224426
S31508001A48D2F814324344C2F8143246E7206801F043
S31508001A58B4FC8046B14617E007EB49130122C3F8E0
S31508001A68082B49462046FFF75DFE1DE007EB49139C
S31508001A780822C3F8082B49462046FFF7D3FE16E086
S31508001A8809F101094FEA5808B8F1000F3FF431AFD8
S31508001A9818F0010FF4D05FFA89F1206801F09DFC6F
S31508001AA8824610F0010FD7D11AF0080FDED11AF0C6
S31508001AB8100F04D007EB49131022C3F8082B1AF0A5
S31508001AC8200F04D007EB49132022C3F8082B1AF471
S31508001AD8005FD5D007EB49134FF40052C3F8082B1B
S31508001AE8CEE7206801F071FC8046B1462AE05946DF
S31508001AF8204603F0EBFB1AF0080F04D007EB49134E
S31508001B080822C3F808291AF0100F04D007EB49135E
S31508001B181022C3F808291AF0400F04D007EB491316
S31508001B284022C3F808291AF0020F04D007EB491314
S31508001B380222C3F808291AF0800F41D109F10109D0
S31508001B484FEA5808B8F1000F3FF4DAAE18F0010F5B
S31508001B58F4D05FFA89FB5946206801F047FC8246AB
S31508001B6810F0010FC7D009F00F03012101FA03F29B
S31508001B78D7F8343823EA0203C7F8343807EB491389
S31508001B88C3F8081923698B42B1D14FEAC902A2EBF7
S31508001B98090293002344596C9A6C0A449A64B9F169
S31508001BA8000FA4D1C9EBC902930023441B6D002B6F
S31508001BB89DD104F571720121206801F03FFC96E772
S31508001BC849462046FFF766FCB8E7D5F8043823F0F7
S31508001BD80103C5F8043894F8F433012B08D02046D5
S31508001BE803F0BAFB2268536903F0004353618DE694
S31508001BF8002184F8F413204600F076FAF2E7204626
S31508001C0803F090FB8EE6204603F08CFBABE605F561
S31508001C180068D8F8043023F00103C8F80430102106
S31508001C28206800F099FF20E007EB46134FF67F314E
S31508001C38C3F80819D3F8002922F40012C3F80029B2
S31508001C48D3F8002942F00062C3F80029C3F8081B34
S31508001C58D3F8002B22F40012C3F8002BD3F8002B74
S31508001C6842F00062C3F8002B01366368B342DBD83A
S31508001C78D8F81C3043F00113C8F81C30236BEBB1B5
S31508001C88D8F8843043F00B03C8F88430D8F84430C1
S31508001C9843F00B03C8F84430D5F8003823F4FE633C
S31508001CA8C5F8003804F57172217C206801F0C6FB76
S31508001CB82268536903F4805353615BE6D8F8142005
S31508001CC842F22B031343C8F81430D8F8103043F0FF
S31508001CD80B03C8F81030DFE7206801F09FFB20687F
S31508001CE801F03AF8E060256800F000FA227B014620
S31508001CF8284600F097FE204603F0FAFA2268536948
S31508001D0803F4005353613CE6204603F0EAFA2268D6
S31508001D18536903F0080353613AE60021204603F0A5
S31508001D282AFB2268536903F48013536137E60021B6
S31508001D38204603F01AFB2268536903F4001353611B
S31508001D4834E6204603F01DFB2268536903F08043F6
S31508001D58536132E6204603F01EFB3BE690F8BC3397
S31508001D68012B0BD010B50446012380F8BC33006854
S31508001D7801F007FB002084F8BC0310BD0220704759
S31508001D8890F8BC33012B0BD010B50446012380F814
S31508001D98BC33006801F001FB002084F8BC0310BDC1
S31508001DA80220704790F8BC33012B0DD010B50446B5
S31508001DB8012380F8BC3380F83810006801F0D1FA9E
S31508001DC8002084F8BC0310BD02207047F8B511F04E
S31508001DD8800F28D101F00F06F500AF1BBC00274677
S31508001DE804F5FC74044404343E460644002586F883
S31508001DF8FD5101F00F012170A260E370627802B10B
S31508001E08E180022B1ED090F8BC33012B1DD0054665
S31508001E18012380F8BC332146006800F0ADFF002096
S31508001E2885F8BC03F8BD01F00F06F500AF1BBC002A
S31508001E3827463834044404343E460644012586F8C1
S31508001E483D50D6E700232371DDE70220EAE738B5D7
S31508001E5811F0800F21D101F00F05EA00541BA300E9
S31508001E681C4603F5FC73034404332546054400223F
S31508001E7885F8FD2101F00F01197090F8BC23012A95
S31508001E881AD00446012280F8BC231946006800F0D7
S31508001E98BBFF002084F8BC0338BD01F00F04E2003C
S31508001EA8151BAB001D463833034404332C4604443B
S31508001EB8012284F83D20DDE70220EDE770B501F040
S31508001EC80F05EE00711B8C0004F5FC740444211DF3
S31508001ED8761BB4000444C4F80822C4F81032002358
S31508001EE8C4F8143284F8FD3184F8FC510369012BCF
S31508001EF806D065B1DAB2006801F094F8002070BD22
S31508001F08C5EBC506B4000444C4F80C22F1E7DAB2F6
S31508001F18006800F0E7FFF1E701F00F01C1EBC10126
S31508001F288B001844D0F81402704770B501F00F05F5
S31508001F38EE00711B8C0038340444211D761BB4004E
S31508001F480444A264236500236365012384F83D30AD
S31508001F5884F83C500369012B06D05DB1DAB20068F3
S31508001F6801F060F8002070BDC5EBC506B40004444E
S31508001F78E264F2E7DAB2006800F0B4FFF2E738B5CF
S31508001F8801F00F0543689D4236D811F0800F20D11D
S31508001F98CA00541AA3001C4603F5FC730344043309
S31508001FA822460244002182F8FD1101229A701D700A
S31508001FB890F8BC23012A21D00446012280F8BC23C4
S31508001FC81946006801F04EF97DB1002084F8BC0373
S31508001FD813E0EA00511B8B001946383303440433CF
S31508001FE80144012281F83D20DFE704F57172217C5E
S31508001FF8206801F023FAE8E7012038BD0220FCE74B
S3150800200810B501F00F0443689C422CD811F0800FD4
S315080020181DD1E3001A1B91000A4601F5FC7101441B
S3150800202804310244002382F8FD3100238B700C70BA
S3150800203890F8BC33012B18D00446012380F8BC332A
S31508002048006801F03CF9002084F8BC030CE0E300C2
S315080020581A1B91000A463831014404310244012307
S3150800206882F83D30E1E7012010BD0220FCE730B4D4
S315080020780468606A29B10D46A36A00EB1340002379
S315080020880CE040EA0240A06212E003F1400104EBCA
S315080020988101496800EB11400133DBB2691E8B42A6
S315080020A8F3D340EA024005F13F0104EB8101486099
S315080020B8002030BC7047036859620020704700004A
S315080020C8024603680121C0F8FC13002082F8F403CD
S315080020D89A6942F000629A61596D024A0A435A653A
S315080020E8704700BF0300001070470000014B1868CE
S315080020F8704700BF00000020534B98421FD0534B2F
S31508002108984228D0524B984231D0524B98423AD0EE
S31508002118514B984243D0514B98424CD0504B984219
S3150800212855D0504B98425ED04F4B984267D04F4B8C
S31508002138984270D04E4B984279D00120704703F5E3
S3150800214860531A6942F001021A611A6922F00102FB
S315080021581A610020704703F550531A6942F00202C3
S315080021681A611A6922F002021A610020704703F5FB
S3150800217840531A6942F004021A611A6922F00402E5
S315080021881A610020704703F530531A6942F00802AD
S315080021981A611A6922F008021A610020704703F5C5
S315080021A820531A6942F010021A611A6922F01002BD
S315080021B81A610020704703F510531A6942F0200285
S315080021C81A611A6922F020021A610020704703F57D
S315080021D800531A6942F040021A611A6922F040024D
S315080021E81A610020704703F5E0531A6942F0800225
S315080021F81A611A6922F080021A610020704703F5ED
S31508002208C0531A6942F480721A611A6922F48072F4
S315080022181A610020704703F5A0531A6942F4007240
S315080022281A611A6922F400721A610020704703F5C8
S3150800223880531A6942F480621A611A6922F4806224
S315080022481A610020704700BF0000024000040240DF
S3150800225800080240000C0240001002400014024028
S3150800226800180240001C02400020024000240240D8
S3150800227800280240F0B40A6892FAA2F2B2FA82F288
S315080022882DE00E69C46893FAA3F5B5FA85F56D00CD
S31508002298032707FA05F524EA050493FAA3F5B5FA18
S315080022A885F56D0006FA05F52C43C4604C68022CC2
S315080022B840D04C68056893FAA3F6B6FA86F676000F
S315080022C8032707FA06F625EA060593FAA3F3B3FAE7
S315080022D883F35B0004FA03F32B43036001320B68AC
S315080022E833FA02F45AD0012494402340F6D04C68B5
S315080022F8013C012CC5D88E68846893FAA3F5B5FA0B
S3150800230885F56D00032707FA05F524EA050493FA07
S31508002318A3F5B5FA85F56D0006FA05F52C4384602C
S315080023280E68CD68446824EA060405FB06F52C43BE
S315080023384460A6E793FAA3F4B4FA84F4072C15D8EC
S315080023484E69046A93FAA3F5B5FA85F5AD000F2721
S3150800235807FA05F524EA050493FAA3F5B5FA85F507
S31508002368AD0006FA05F52C430462A2E74D69466AEC
S315080023781C0A94FAA4F7B7FA87F7BF004FF00F0CB0
S315080023880CFA07F726EA070694FAA4F4B4FA84F4CA
S31508002398A40005FA04F4344344628AE70020F0BC32
S315080023A87047000082B0224A136843F0010313609D
S315080023B81F4B1B6813F0020FFAD01D4B00229A60B8
S315080023C81A68019201991B4A0A400192019A1A60F1
S315080023D81A6822F0F80242F080021A60144B1B6849
S315080023E813F0007FFAD1124B1B6813F0006FFAD16D
S315080023F80F4B1B6813F0005FFAD10D4B0E4A5A6053
S31508002408103AC3F88420C3F88820DA6822F4FE4212
S31508002418DA60DA6842F47F02DA605A6F22F001025B
S315080024285A675A6F42F080725A67002002B070479E
S3150800243800380240FFFFF2EA10300024034B9B687D
S31508002448C3F30313024AD35CD840704700380240E6
S315080024587C550008034B9B68C3F38223024AD35C66
S31508002468D8407047003802408C550008034B9B68D3
S31508002478C3F34233024AD35CD84070470038024057
S315080024888C5500080D4B5B6803F480030BB90C48A0
S3150800249800E00C48094A536803F03F03B0FBF3F31E
S315080024A85068C0F3881000FB03F05368C3F3014370
S315080024B801335B00B0FBF3F0704700BF00380240F9
S315080024C80024F40000127A0008B5074B9B6803F04D
S315080024D80C03042B06D0082B01D0044808BDFFF7C7
S315080024E8D1FFFBE70248F9E7003802400024F40068
S315080024F800127A0010B50446FFF7E6FF2060FFF7DA
S315080025089DFF6060FFF7A6FFA0606068FFF7AEFF53
S31508002518E06010BD08B5032808D00C282DD0B0F502
S31508002528406F51D0302877D0002008BD584BD3F8D3
S315080025389030034043EA0040564B98420FD0B0F11A
S31508002548031F13D0013B984206D0FFF7BDFFFFF7DC
S3150800255875FFFFF78BFFE8E7FFF7B6FFE5E74C4B94
S315080025681B6813F0020F7ED10020DEE7484B1B6F6D
S3150800257813F0020F79D10020D7E7454BD3F89030EE
S31508002588034043EA0040444B98420FD0B0F10C1F71
S3150800259813D0043B984206D0FFF796FFFFF74EFF85
S315080025A8FFF758FFC1E7FFF78FFFBEE7384B1B68F1
S315080025B813F0020F5CD10020B7E7354B1B6F13F0F9
S315080025C8020F57D10020B0E7314BD3F890300340BB
S315080025D843EA0040314B984210D0B0F10C2F14D082
S315080025E8A3F58063984206D0FFF76EFFFFF726FF2C
S315080025F8FFF73CFF99E7FFF767FF96E7244B1B6849
S3150800260813F0020F39D100208FE7214B1B6F13F007
S31508002618020F34D1002088E71D4BD3F890300340C9
S3150800262843EA00401E4B98420FD0B0F1301F13D032
S31508002638103B984206D0FFF747FFFFF7FFFEFFF764
S3150800264809FF72E7FFF740FF6FE7114B1B6813F0A6
S31508002658020F17D1002068E70D4B1B6F13F0020F06
S3150800266812D1002061E70F485FE74FF400405CE7A6
S315080026780C485AE74FF4004057E70A4855E74FF41D
S31508002688004052E7074850E74FF400404DE700BFBF
S31508002698003802400200030008000C000008000C7D
S315080026A8200030000024F40008B5C0280AD0B0F588
S315080026B8407F2FD0B0F5405F54D0B0F5404F79D061
S315080026C8002008BD594BD3F89030034043EA004030
S315080026D8574B98420FD0B0F1C01F14D0403B9842D0
S315080026E806D0FFF7F1FEFFF7A9FEFFF7B3FEE8E706
S315080026F8FFF7EAFEE5E74D4B1B6813F0020F40F0BB
S3150800270881800020DDE7494B1B6F13F0020F7BD150
S315080027180020D6E7454BD3F89030034043EA0040FB
S31508002728444B984210D0B0F1032F14D0A3F5807308
S31508002738984206D0FFF7C8FEFFF780FEFFF78AFE25
S31508002748BFE7FFF7C1FEBCE7384B1B6813F0020F5B
S315080027585DD10020B5E7354B1B6F13F0020F58D132
S315080027680020AEE7314BD3F89030034043EA0040E7
S31508002778314B984210D0B0F1302F14D0A3F58053BE
S31508002788984206D0FFF7A0FEFFF758FEFFF762FE4D
S3150800279897E7FFF799FE94E7244B1B6813F0020F97
S315080027A83AD100208DE7214B1B6F13F0020F35D164
S315080027B8002086E71D4BD3F89030034043EA0040D3
S315080027C81E4B984210D0B0F1C02F14D0A3F5804301
S315080027D8984206D0FFF778FEFFF730FEFFF73AFE75
S315080027E86FE7FFF771FE6CE7104B1B6813F0020FD3
S315080027F817D1002065E70D4B1B6F13F0020F12D196
S3150800280800205EE70E485CE74FF4004059E70C489D
S3150800281857E74FF4004054E7094852E74FF4004099
S315080028284FE707484DE74FF400404AE700380240AB
S315080028388000C0000002000300200030008000C0AD
S315080028480024F40038B5036813F0010F75D10D4656
S31508002858044603683C4A1A404B68C9680B43296909
S315080028680B43A9690B4313430360AB68426822F418
S315080028784052134343606B69826822F440721343DB
S315080028888360324B984216D0314B984227D0314B49
S31508002898984228D0304B984229D0304B98422AD0B3
S315080028A82F4B98422CD02F4B98422ED02E4B98421D
S315080028B830D0012042E00320FFF72CFE00283ED046
S315080028C82B68002B3DD0AA69B2F5004F27D000EB3C
S315080028D85300B0FBF3F080B2E06000202EE00C2035
S315080028E8FFF718FEEAE73020FFF714FEE6E7C020F0
S315080028F8FFF7DAFEE2E74FF44070FFF7D5FEDDE7AB
S315080029084FF44060FFF706FED8E74FF44050FFF74C
S31508002918CBFED3E74FF44040FFF7C6FECEE75A088A
S3150800292802EB4000B0FBF3F04FF6F0730340C0F338
S3150800293842001843E060002000E0012038BD01206D
S31508002948FCE70120FAE700BFF369FFEF0010014032
S315080029580044004000480040004C00400050004039
S315080029680014014000780040007C00400023013331
S315080029780C4A934211D80269002AF8DA036943F027
S315080029880103036100230133064A934207D8026903
S3150800299812F0010FF7D10020704703207047032073
S315080029A8704700BF400D030084B010B5044603A85D
S315080029B880E80E00089B012B1DD1A36B23F48033F6
S315080029C8A363E268164B1340E360E36823F44013F5
S315080029D8E3600F9B012B09D02046FFF7C7FF069B2C
S315080029E8012B14D0BDE8104004B07047E36843F4DF
S315080029F88013E360F0E7E36843F04003E3602046AA
S31508002A08FFF7B4FFA36B43F48033A363E7E7A36830
S31508002A1843F00603A360A36843F02003A360E1E735
S31508002A28BFFFBDFF022A0AD00921C26822F47052E4
S31508002A38C260C36843EA8123C36000207047274BF6
S31508002A480B44274A934239D9264B0B44264A9342C4
S31508002A5836D9264B0B44264A934233D9254B0B4481
S31508002A6802F5C332A03293422ED9234B0B44234A8C
S31508002A7893422BD9224B0B4402F5922202F578721F
S31508002A88934225D91F4B0B4402F5C32202F520723F
S31508002A9893421FD91C4B0B4402F5B71202F558721C
S31508002AA8934219D9194B0B4402F5122202F5F8621A
S31508002AB8934201D90621B8E70721B6E70F21B4E7FB
S31508002AC80E21B2E70D21B0E70C21AEE70B21ACE7E2
S31508002AD80A21AAE70921A8E70821A6E7405327FFFC
S31508002AE8FF340C00401E1BFF3F420F0000DC0BFFA3
S31508002AF87F4F1200808CF9FE60B6E5FE5FE316008C
S31508002B0800D3CEFEC05BB3FE00CA91FEE05459FE60
S31508002B18836843F00103836000207047836823F0C5
S31508002B28010383600020704708B5C36823F0C043D3
S31508002B38C360012909D069B9C36843F08043C360F3
S31508002B483220FDF771FE002008BDC36843F0005324
S31508002B58C360F5E70120F7E7890141F02001016123
S31508002B6800230133054A934205D8026912F0200F5B
S31508002B78F7D1002070470320704700BF400D0300B7
S31508002B881023036100230133054A934205D80269D5
S31508002B9812F0100FF7D1002070470320704700BFC6
S31508002BA8400D0300D0F800381943C0F80018002073
S31508002BB87047000084B02DE9F041044607A880E86C
S31508002BC80E002546002306E003F1400204EB8202C4
S31508002BD80021516001330E2BF6D9119B33BBD4F86B
S31508002BE8043843F00203C4F80438A36B23F400132B
S31508002BF8A363236843F040032360236843F08003F4
S31508002C0823600023C4F8003E04F50066D4F80038AB
S31508002C18C4F800380C9B012B0DD0032B1CD1099B3B
S31508002C28ABB900212046FFF7BDFF19E0A36B43F4B3
S31508002C380013A363E5E7099B23B900212046FFF79C
S31508002C48B1FF0DE001212046FFF7ACFF08E001219E
S31508002C582046FFF7A7FF03E003212046FFF7A2FF58
S31508002C6810212046FFF778FF804608B14FF0010883
S31508002C782046FFF785FF08B14FF0010800233361A6
S31508002C887361F3610AE0C3B94FF00060C2F800093E
S31508002C9800220A614FF67F328A6001330799994202
S31508002CA810D905EB431202F51061D2F8000900287D
S31508002CB8E9DB0020C2F80009EAE74FF09040C2F8BD
S31508002CC80009E5E700230AE0BBB14FF09047C2F8D0
S31508002CD8007B002202614FF67F32826001339942F7
S31508002CE810D905EB431202F53060D2F8007B002FA5
S31508002CF8EADB0027C2F8007BEBE74FF00067C2F86B
S31508002D08007BE6E7336923F4807333610023A36104
S31508002D186FF0804363610A9B1BB9A36943F01003EC
S31508002D28A361A2690A4B1343A3610D9B1BB1A3694F
S31508002D3843F00803A361119B012B04D04046BDE864
S31508002D48F04104B07047A269024B1343A361F5E743
S31508002D5800383C8004000040D0F8083813F0060311
S31508002D6805D0062B18BF022B03D102207047002076
S31508002D7870470F207047000070B40B784A78012A0C
S31508002D8820D0D0F81C2803F00F060124B44042EAE4
S31508002D980442C0F81C2800EB4310D0F8003B13F493
S31508002DA8004F0CD1D0F8002B8B68C3F30A03C978F7
S31508002DB843EA81431343134A1A43C0F8002B0020F9
S31508002DC870BC7047D0F81C4803F00F06B24092B2A0
S31508002DD82243C0F81C2800EB4310D0F8002912F447
S31508002DE8004FECD1D0F800498A68C2F30A02C978BC
S31508002DF842EA814242EA83532343024A1A43C0F805
S31508002E080029DCE70080001030B40B784A78012ADC
S31508002E1824D000EB4313D3F8002B002A50DBD0F854
S31508002E283C580A7802F00F02012404FA02F225EA4D
S31508002E380242C0F83C28D0F81C28097801F00F018E
S31508002E488C4022EA0444C0F81C48D3F8001B234ADD
S31508002E580A40C3F8002B002030BC704700EB431328
S31508002E68D3F80029002A1EDBD0F83C580A7802F065
S31508002E780F02012404FA02F292B225EA0202C0F805
S31508002E883C28D0F81C28097801F00F018C40A4B218
S31508002E9822EA0404C0F81C48D3F80019104A0A4064
S31508002EA8C3F80029D7E7D3F8002942F00062C3F827
S31508002EB80029D3F8002942F08042C3F80029D3E74D
S31508002EC8D3F8002B42F00062C3F8002BD3F8002B86
S31508002ED842F08042C3F8002BA1E700BF0078F3EF61
S31508002EE8007833EC70B40B784C78012C24D000EBBE
S31508002EF8431000F530631D693E4C2C401C611D6962
S31508002F083D4C2C401C614C690CB18C684C611C69A1
S31508002F1844F400241C611C698D68C5F312052C430A
S31508002F281C61012A61D0D0F8003B43F00443C0F87D
S31508002F38003B002070BC70474C695CBB00EB43142F
S31508002F48D4F810692C4D3540C4F81059D4F81059DE
S31508002F5845F40025C4F81059D4F81069254D3540AC
S31508002F68C4F81059012A31D000EB4313D3F80029C5
S31508002F7842F00442C3F800294B69002BD9D0D0F88F
S31508002F883428097801F00F040121A1400A43C0F842
S31508002F983428CEE700EB431404F510642669154D6A
S31508002FA8354025612669144D354025614E698D6879
S31508002FB8AE4200D94D61256945F400252561256984
S31508002FC84E69C6F3120635432561CBE70A691AB175
S31508002FD800EB4311C1F8142900EB4310D0F8002977
S31508002FE842F00442C0F80029A3E7CA68002A9AD022
S31508002FF85A6198E70000F8FFFFFF07E070B49DF8EC
S315080030080C4064B903339D0807E000EB023303F567
S31508003018805351F8046B1E600134AC42F5D3002086
S3150800302870BC7047F0B583B00B784C78012C29D062
S3150800303800EB431303F5306426697D4D3540256159
S3150800304826697C4D354025614D69002D40F0C180C3
S3150800305825698E68C6F3120635432561256945F440
S3150800306800252561012A00F0C980CA78012A00F0DE
S31508003078CB80D3F8002B42F00442C3F8002B00207B
S3150800308803B0F0BD4C6974BB00EB4314D4F810695F
S31508003098684D3540C4F81059D4F8105945F4002538
S315080030A8C4F81059D4F81069614D3540C4F8105958
S315080030B8012A4AD000EB4313D3F8004944F00444E4
S315080030C8C3F80049CC78012C68D04B69002BD6D0B8
S315080030D8D0F83428097801F00F040121A1400A43E1
S315080030E8C0F83428CBE700EB4314D4F81069504DE0
S315080030F83540C4F81059D4F810694E4D3540C4F80F
S315080031081059D4F810694D698F683D44013DB5FBDF
S31508003118F7F5494F07EAC5453543C4F81059D4F8B1
S3150800312810594E69C6F312063543C4F8105904F502
S315080031381064CD78012DBBD1256925F0C0452561D8
S31508003148256945F000552561B2E70A691AB100EB09
S315080031584314C4F81429CA78012A08D000EB431383
S31508003168D3F8002942F00442C3F8002987E7D0F8C3
S31508003178082812F4807F08D100EB4311D1F80029FA
S3150800318842F00052C1F80029E8E700EB4311D1F8EC
S31508003198002942F08052C1F80029DFE7D0F808482C
S315080031A814F4807F0ED1D3F8004944F00054C3F8CC
S315080031B8004914460B46C9681A789B8A0094FFF793
S315080031C81DFF5CE7D3F8004944F08054C3F800496A
S315080031D8EFE78E683544013DB5FBF6F52669164FC7
S315080031E807EAC5473E43266127698E68ADB206FBDE
S315080031F805F5C5F312053D43256133E7CA68002A74
S315080032083FF433AF626130E7D0F8082812F4807FBC
S3150800321806D1D3F8002B42F00052C3F8002B28E752
S31508003228D3F8002B42F08052C3F8002B21E700BFE1
S315080032380000F8FFFFFF07E00000F81F03329208B6
S31508003248002393420CD210B400F58054246841F840
S31508003258044B01339342F7D308465DF8044B70478D
S31508003268084670470B784A78012A14D000EB4310B1
S31508003278D0F8002B002A06DB2BB1D0F8003B23F048
S315080032888043C0F8003BD0F8003B43F40013C0F86D
S31508003298003B0020704700EB4310D0F80029002AAD
S315080032A806DB2BB1D0F8003923F08043C0F8003983
S315080032B8D0F8003943F40013C0F80039E9E70B7869
S315080032C84A78012A0ED000EB4310D0F8003B23F4C5
S315080032D80013C0F8003BCB78023BDBB2012B15D9AB
S315080032E80020704700EB4310D0F8003923F4001388
S315080032F8C0F80039CB78023BDBB2012BF0D8D0F8FE
S31508003308003943F08053C0F80039E9E7D0F8003BA4
S3150800331843F08053C0F8003BE2E738B50546044653
S31508003328002208E004EB42134FF67F31C3F8081968
S31508003338C3F8081B01320E2AF4D90022C5F810284A
S31508003348C5F81428C5F81C282846FFF719FC0346AB
S3150800335808B1184638BD10212846FFF7FDFB034675
S31508003368F7E7D0F8003823F4FE63C0F80038D0F839
S315080033780038090101F4FE610B43C0F80038002043
S31508003388704708B5D0F8043823F00203C0F80438A3
S315080033980320FDF749FA002008BD08B5D0F8043817
S315080033A843F00203C0F804380320FDF73DFA00206D
S315080033B808BD4269806910407047D0F8183800F58A
S315080033C80060C0691840000C7047D0F8183800F536
S315080033D80060C069184080B2704700EB4111D1F807
S315080033E8082B00F5006040691040704710B4D0F803
S315080033F81048D0F8343801F00F02D340DB01DBB2AD
S31508003408234300EB411000F51060806818405DF80A
S31508003418044B7047406900F001007047D0F800294E
S31508003428054B1340C0F80039D0F8043843F48073C4
S31508003438C0F804380020704700F8FFFF10B4046C81
S31508003448154B9C4203D9D0F8003B002B16DB002409
S31508003458C0F8104BD0F8104B44F40024C0F8104BB1
S31508003468D0F8104B44F01804C0F8104BD0F8104B9D
S3150800347844F0C044C0F8104B012903D000205DF879
S31508003488044B7047C0F8142BD0F8003B43F0802350
S31508003498C0F8003BF2E700BF0A30544F014B1860EA
S315080034A8704700BF00000020C0B108B50346D0F831
S315080034B8B80210B10020C3F8B802D3F8CC0210B18C
S315080034C80020C3F8CC0209B1C3F8B4121846012380
S315080034D880F89C32027001F069FF08BD0320704726
S315080034E810B50446012380F89C32D0F8B83213B1D7
S315080034F85B6801799847D4F8CC3213B10023C4F82D
S31508003508CC32204601F0C2FF034608B1184610BD62
S31508003518204601F0ABFF0346F8E710B582B0002352
S31508003528ADF8063059B10446C4F8B812CB6A0DF19D
S3150800353806009847C4F8CC02002002B010BD032044
S31508003548FBE708B501F09AFF08BD08B5D0F8B83208
S3150800355813B11B68984708BD0320FCE708B5D0F8DF
S31508003568B8320BB15B689847002008BD38B50446E1
S3150800357800F2AA25284600F02DF90123C4F894324A
S31508003588B4F8B032C4F8983294F8AA1201F01F03B6
S31508003598012B0DD03BB1022B0FD001F0800120463C
S315080035A801F08FFF03E02946204600F0CEFA38BD21
S315080035B82946204600F004FBF9E72946204600F08C
S315080035C833FBF4E710B5044629BB1346D0F8942212
S315080035D8032A01D0002029E0D0F85C11D0F8602130
S315080035E891420DD8D0F8B8321B6923B190F89C22BD
S315080035F8032A00D19847204600F067FC002015E00A
S31508003608891AC0F85C118A4228BF0A46194600F08A
S3150800361854FC00200AE00A46D0F8B8329B6933B150
S3150800362890F89C12032904D11146984710BD032027
S31508003638FCE70320FAE710B50446002946D11346E5
S31508003648D0F89422022A05D094F8A032012B39D052
S31508003658002046E0C269016A8A4213D88A421DD008
S31508003668D4F8B832DB682BB194F89C22032A01D126
S31508003678204698478021204601F023FF204600F07F
S315080036882FFCE1E7521AC261194600F00EFC002326
S315080036981A461946204601F034FFD5E78369994248
S315080036A8DED8D0F898229342DAD20022114600F0E2
S315080036B8FCFB0021C4F898120B460A46204601F07E
S315080036C820FFC1E7002084F8A0020AE00A46D0F8DD
S315080036D8B8325B6933B190F89C12032904D11146B4
S315080036E8984710BD0320FCE70320FAE770B504469F
S315080036F8012380F89C320023C0F894324360C0F84E
S31508003708A432D0F8BC3223B1D0F8B8325B680021AD
S315080037189847402300221146204601F0BFFE01269D
S31508003728A4F864614025C4F860512B46002280211C
S31508003738204601F0B3FEA6842562002070BD0174F8
S315080037480020704790F89C3280F89D32042380F850
S315080037589C320020704790F89C32042B01D0002038
S31508003768704790F89D3280F89C32F8E708B590F8CB
S315080037789C32032B01D0002008BDD0F8B832DB698B
S31508003788002BF8D09847F6E70020704700207047C6
S315080037980020704708B5012380F89C32D0F8B83263
S315080037A813B15B6801799847002008BD002302E039
S315080037B80133DBB201300278002AF9D1184670477E
S315080037C808B54B88012B00D008BDC0F8A43200F014
S315080037D87CFBF9E70B7803704B7843708B78CA78CB
S315080037E843EA022343800B794A7943EA0223838012
S315080037F88B79CA7943EA0223C380704710B5044611
S31508003808802101F05EFE0021204601F05AFE10BD17
S3150800381830B583B004460D460023ADF806304A880D
S31508003828130A013B062B00F2AB80DFE803F0041FFE
S3150800383833A9A98D9A00D0F8B4321B680DF1060190
S31508003848007C9847EA88002A00F0A380BDF806306D
S31508003858002B00F099809A4228BF1A46ADF8062030
S315080038680146204600F014FB03B030BD037C43B97B
S31508003878D0F8B8329B6A0DF10600984702234370C0
S31508003888E0E7D0F8B832DB6A0DF10600984702235C
S315080038984370D7E7D2B2052A52D8DFE802F00310F8
S315080038A81D2A3744D0F8B4325B6823B10DF10601F6
S315080038B8007C9847C6E72946FFF7A0FFD4E7D0F863
S315080038C8B4329B6823B10DF10601007C9847B9E725
S315080038D82946FFF793FFC7E7D0F8B432DB6823B168
S315080038E80DF10601007C9847ACE72946FFF786FFE5
S315080038F8BAE7D0F8B4321B6923B10DF10601007C8A
S3150800390898479FE72946FFF779FFADE7D0F8B4321D
S315080039185B6923B10DF10601007C984792E72946B1
S31508003928FFF76CFFA0E7D0F8B4329B6923B10DF115
S315080039380601007C984785E72946FFF75FFF93E766
S315080039482946FFF75BFF8FE7037C33B9D0F8B8320F
S315080039585B6B0DF10600984774E72946FFF74EFF9B
S3150800396882E7037C43B9D0F8B8321B6B0DF1060021
S3150800397898470723437065E72946FFF73FFF73E72C
S315080039882946FFF73BFF6FE729462046FFF736FF2C
S315080039986AE7204600F099FA66E738B504468B8840
S315080039A8F3B9CB88E3B94B887F2B19D803F07F0581
S315080039B890F89C32032B0CD080F89E52294601F0C9
S315080039C890FD204600F081FA35B1022384F89C322E
S315080039D809E0FFF713FF06E0012384F89C3202E0AA
S315080039E82046FFF70BFF38BD70B504460D468978A3
S315080039F82E4B197001290FD890F89C32022B11D03A
S31508003A08032B25D02946FFF7F9FE284B19782046B7
S31508003A18FFF7A4FD032603E02946FFF7EFFE032672
S31508003A28304670BD81B14160FFF78FFD064620B16B
S31508003A3829462046FFF7E2FEF2E7204600F045FA57
S31508003A48032384F89C32EBE700F03FFA0026E7E701
S31508003A58C9B14368994225D0D9B2FFF77FFD134B00
S31508003A68197861602046FFF770FD0646B0B1294609
S31508003A782046FFF7C3FE21792046FFF76FFD02238C
S31508003A8884F89C32CCE7022380F89C324160FFF721
S31508003A9865FD204600F019FA0026C1E7204600F021
S31508003AA814FABDE700F011FA0026B9E7E800002085
S31508003AB808B5CB88012B0BD190F89C329BB1022B09
S31508003AC809D9032B0FD10122011D00F0E1F901E004
S31508003AD8FFF794FE08BD0146002341F8083F012276
S31508003AE800F0D6F9F6E7FFF789FEF3E708B590F888
S31508003AF89C32013B022B12D8CB88022B0CD101230E
S31508003B08C360D0F8A4320BB10323C360022200F1C4
S31508003B180C0100F0BDF908BDFFF770FEFBE7FFF7DB
S31508003B286DFEF8E708B590F89C32013B022B09D8D8
S31508003B384B88012B00D008BD0023C0F8A43200F03A
S31508003B48C4F9F8E7FFF75AFEF5E708B50B7803F066
S31508003B586003202B06D0402B04D043B1FFF74EFE56
S31508003B68002003E0D0F8B8329B68984708BD4B7820
S31508003B78092B21D8DFE803F0141C20182009052092
S31508003B88100DFFF745FE0020F0E7FFF706FF0020B7
S31508003B98ECE7FFF729FFE9E7FFF78AFF0020E5E7E3
S31508003BA8FFF7A4FF0020E1E7FFF70AFE0020DDE79C
S31508003BB8FFF7B8FF0020D9E7FFF720FE0020D5E772
S31508003BC870B505460C460B7803F06003202B07D022
S31508003BD8402B05D023B1FFF711FE0026304670BDED
S31508003BE895F89C32013B022B18D82379012B0FD85C
S31508003BF8D5F8B8329B682146284698470646E3888A
S31508003C08002BEBD10028E9D1284600F05EF9E5E754
S31508003C1821462846FFF7F2FD0026DFE72146284613
S31508003C28FFF7ECFD0026D9E738B505460C468A881D
S31508003C380B7803F06003202B08D0D1B2402B05D0AF
S31508003C485BB12146FFF7DAFD002005E0D5F8B83262
S31508003C589B6821462846984738BD6378012B38D093
S31508003C68002B6BD0032B40F0F08090F89C32022B87
S31508003C7806D0032B19D02146FFF7C0FD0020EBE735
S31508003C88B1F1800318BF0123002908BF00233BB1FF
S31508003C9801F017FC8021284601F013FC0020DBE719
S31508003CA82146FFF7ABFD0020D6E763884BB9B1F18B
S31508003CB8800318BF0123002908BF00230BB1E38836
S31508003CC823B1284600F001F90020C5E701F0F9FB01
S31508003CD8F7E790F89C32022B06D0032B19D0214619
S31508003CE8FFF78CFD0020B7E7B1F1800318BF012361
S31508003CF8002908BF00233BB101F0E3FB80212846D1
S31508003D0801F0DFFB0020A7E72146FFF777FD002033
S31508003D18A2E76388002B40F09D8011F07F0F0AD137
S31508003D28284600F0D2F8D5F8B8329B6821462846C6
S31508003D389847002090E701F0CCFBF1E790F89C3211
S31508003D48022B06D0032B2FD02146FFF757FD00205C
S31508003D5882E7B1F1800318BF0123002908BF0023B1
S31508003D689BB912F0800F15D101F07F0101EB810193
S31508003D788B0003F5A8710144043100240C60022263
S31508003D88284600F085F8204666E72146FFF736FDFF
S31508003D98002061E701F07F0101EB81018B0003F147
S31508003DA8100101440431E8E752B2002A24DB01F085
S31508003DB80F0303EB830398002844B0F8643153B320
S31508003DC8002A2EDB01F07F0202EB8202930003F53C
S31508003DD8A8742C440434802914BF0023012300291D
S31508003DE808BF01233BB30023236002222146284645
S31508003DF800F04EF800202FE701F00F0303EB8303CA
S31508003E0898002844838C002BDAD121462846FFF7E8
S31508003E18F5FC002020E721462846FFF7EFFC00209E
S31508003E281AE701F07F0202EB8202930003F11004FD
S31508003E382C440434CFE7284601F0F2FA10B10123DE
S31508003E482360D2E700232360CFE72146FFF7D6FC95
S31508003E58002001E70020FFE6C8B170B50D461646F2
S31508003E680446FFF7A3FC013040003080287003237E
S31508003E786B70022307E0EA5401345A1CD2B20021B7
S31508003E88A9540233DBB22278002AF4D170BD7047F0
S31508003E9810B513460222C0F894228361C3610A4604
S31508003EA8002101F026FB002010BD08B513460A4676
S31508003EB8002101F01EFB002008BD08B513460A4676
S31508003EC8002101F01EFB002008BD08B50423C0F830
S31508003ED8943200231A46194601F00BFB002008BD48
S31508003EE808B50523C0F8943200231A46194601F086
S31508003EF808FB002008BD72B6704762B67047000016
S31508003F082DE9F04184B004460D461746984668469A
S31508003F18FEF7F0FA0299164BA3FB0131890900222C
S31508003F2801E00132D2B2112A1DD8124B13F8120039
S31508003F3803EB420393F801C000EB0C0303FB0443AD
S31508003F48B1FBF3FE03FB1E16002EEAD11FFA8EF309
S31508003F582B80013B9BB2B3F5806FE2D2387088F8A4
S31508003F6800C0012000E0002004B0BDE8F08100BFD1
S31508003F78D34D6210D055000870B58CB00022ADF844
S31508003F882E208DF82D200CAB03F8042D0DF12D02EB
S31508003F980DF12E014FF4FA70FFF7B2FF002835D05D
S31508003FA81D4C1E4B2360002525766576A5760126C9
S31508003FB8E67625776577A560E5609DF82D30013B9F
S31508003FC81B0423619DF82C30013B1B056361BDF872
S31508003FD82E3063602046FCF73BFC06950795089645
S31508003FE84CF6E043019302954FF6E07303930423D6
S31508003FF80493059509960E230A9301A92046FCF70A
S31508004008CDFC2046FCF760FD0CB070BDB521044810
S3150800401800F034FDC4E700BFEC000020006400404F
S315080040289455000810B588B040F2E173029300234E
S3150800403804930593069101AB024602A90B48FCF7BF
S3150800404871FD08B108B010BD00F028FB00F1320474
S3150800405801990648FCF7DBFD0028F3D000F018FEA6
S3150800406800F01CFBA042F3D9ECE700BFEC000020E7
S3150800407810B588B00C46034601AA00210A48FCF781
S31508004088D8FD60B9019A40F267639A4201D00020C8
S3150800409806E0039B33B9059B2370012000E0002046
S315080040A808B010BD0020FBE7EC00002008B5FFF7B4
S315080040B822FF08BD10B500F0FFF900B910BDFCF7DE
S315080040C8ABF80028FAD000F08DFDFCF759FB00F094
S315080040D8BBFA00F0F5F9054B0340054A936000F072
S315080040E8EFF94468FFF709FFA047E7E780FFFF1FD6
S315080040F800ED00E070B508E04D1C461C0B7803700F
S3150800410800F0C6FD304629462246531E9CB2002AB0
S31508004118F2D170BD38B50546002401E00134E4B291
S31508004128062C15D800F0B4FD04EB44029300094A9E
S31508004138D358AB42F2D804EB44029100054A0A4424
S3150800414852681344AB42E9D9024B0B44187A00E08B
S31508004158FF2038BDF455000808B5C1F3080353B95C
S3150800416803688B4209D040F8041B4FF40072FFF726
S31508004178C1FF012000E0002008BD0120FCE72DE969
S31508004188F0410746FCF7D6FE00247F2C14D83E6873
S31508004198A30006EB03083B445D6800F079FD2A4650
S315080041A8002341460220FCF71BFF38B956F824308D
S315080041B8AB4209D10134E8E7012400E00024FCF702
S315080041C8D1FE2046BDE8F0810024F8E738B50D464B
S315080041D80C4B984211D004460B4B994207D1094C0F
S315080041E829462046FFF7B8FF48B1204638BDFFF7ED
S315080041F8C6FF0028F4D10024F7E7044CF0E70024AA
S31508004208F3E700BF18030020008000081401002007
S315080042182DE9F04106460C4617461D46DFF8748018
S3150800422801EA08080368B3F1FF3F07D03368434536
S315080042380BD13368E41A3444043415E04146FFF7D1
S315080042488BFF03460028F1D11FE041463046FFF7A9
S31508004258BDFF06460028ECD1002316E017F8013BF7
S3150800426804F8013B013D0FD000F012FD331DE31A97
S31508004278B3F5007FF2D308F500713046FFF7A6FFBD
S31508004288064628B1041DE9E701231846BDE8F0816A
S315080042980023FAE700FEFFFF70B586B004460E460F
S315080042A800230193884219D80125ECB1072E1FD897
S315080042B8DDB1002302930223059301230493FCF737
S315080042C839FEB4420DD800F0E3FC039401A902A80C
S315080042D8FCF70AFF20B90134E4B2F2E70025E4E75F
S315080042E80025FCF73FFE00E00025284606B070BD0D
S315080042F80025FAE74FF0FF33024A1360024A1360B3
S31508004308704700BF140100201803002070B54B1E23
S31508004318144C241AA34201D9002070BD16460D462E
S315080043280446FFF7F7FEFF2818D028190138FFF7C3
S31508004338F1FEFF2814D00C4B23400C4A934206D0B2
S315080043482B46324621460A48FFF762FFE5E72B4621
S31508004358324621460748FFF75BFFDEE70020DCE721
S315080043680020DAE7FFFF0F0800FEFFFF00800008BD
S3150800437814010020180300204A1E0D4B1B1A9A42E6
S3150800438801D90020704770B50C460546FFF7C2FEEE
S31508004398064660190138FFF7BDFEFF2818BFFF2E2D
S315080043A801D1002070BD01463046FFF775FFF9E7D1
S315080043B8FFFF0F08104B1B68B3F1FF3F1AD000B573
S315080043C883B00D4A536891680B44D1680B44116948
S315080043D80B4451690B4491690B44D26913445B42F7
S315080043E802AA42F8043D04210448FFF78FFF03B0E8
S315080043F85DF804FB0120704718030020C8810008EF
S315080044080D4B1B680D4A12681A440D4B1B6813445A
S315080044180C4A126813440C4A12681A440B4B1B6858
S315080044281A440B4B1B6813440A4A1268DA4201D02D
S3150800443800207047012070470080000804800008A3
S31508004448088000080C8000081080000814800008FE
S3150800445818800008C881000808B50D4B1B68B3F119
S31508004468FF3F0BD10B4B1B68B3F1FF3F0DD0094833
S31508004478FFF785FE034648B1012307E00448FFF71E
S315080044887EFE03460028EDD100E00123184608BD44
S31508004498180300201401002000487047008000080F
S315080044A808B5FFF727FF08BD08B5FFF72FFF08BDB2
S315080044B808B5FFF761FF08BD08B5FFF7A1FF08BDF6
S315080044C808B5FFF7E9FF08BD08B5FFF773FF034608
S315080044D808B9184608BDFFF7BFFF0346F9E7000005
S315080044E8054BDB6913F0200F04D0034B5B6A037096
S315080044F801207047002070470048004010B5094B56
S31508004508986200F0CBF800F10A04064BDB6913F051
S31508004518800F05D100F0BCFB00F0C0F8A042F4D922
S3150800452810BD00BF0048004010B588B00C4C236881
S3150800453823F0010323604FF4614301930023029398
S31508004548039304930C2205920693079301A9204620
S31508004558FEF778F9236843F00103236008B010BD15
S315080045680048004070B506460D46402904D8284636
S31508004578FFF7C4FF00240BE08321074800F07EFA02
S31508004588F5E700F085FB305DFFF7B8FF0134A4B204
S31508004598ABB2A342F5D870BD4856000870B5254B8E
S315080045A81C78BCB92448FFF79BFF012801D0204690
S315080045B870BD214B1B78013BDBB23F2BF7D800F0C7
S315080045C86DF81E4B18601E4B00221A70194B0122F3
S315080045D81A70ECE706460D46194B1B780133164840
S315080045E81844FFF77DFF0446012815D1144B1A789D
S315080045F80132D2B21A70104B1B789A4201D00024A5
S31508004608D5E710493046FFF775FD0A4B00221A70A0
S315080046180B4B1B782B70CAE700F040F8074B1B6852
S315080046286433984203D90024024B1C70BFE7002460
S31508004638BDE700BF5D0500201C05002060050020B9
S315080046485E0500201D050020024B00221A605A60EC
S315080046589A60704710E000E008B5FFF7F5FF054BCC
S31508004668054A5A6000229A6005211960034B1A60A8
S3150800467808BD00BF10E000E0BF4B0300640500203A
S31508004688044B1B6813F4803F03D0034A13680133AD
S315080046981360704710E000E06405002008B5FFF7CE
S315080046A8EFFF014B186808BD6405002008B5FFF739
S315080046B8F5FF08BD094B03F11801002232B19A74B7
S315080046C800225A61064B054A1A6070479A7459615E
S315080046D8183318310132D2B2F0E700BFA805002016
S315080046E8D80500200A4B1B6883B110B45C69084AD0
S315080046F8146019749860D86000225A7418600139D1
S3150800470808445860987C5DF8044B7047FF2070474A
S31508004718D805002038B504460D4601281CD862007D
S315080047282244D100114B0B445A7C1B7C9A4219D05F
S315080047380E4B0B44DA6815705A7C01325A74DA68DB
S315080047480132DA605B689A420ED9084A0846515817
S315080047580244D160012038BD4FF4E071044800F0E6
S315080047688DF9DCE70020F6E70120F4E7A805002024
S315080047788856000808B50146024B1878FFF7CAFF9D
S3150800478808BD00BFDC05002038B504460D460128DB
S315080047981ED804EB4403DA00124B13445B7CEBB1D6
S315080047A862002244D1000F4B0B449A6812782A708B
S315080047B85A7C013A5A749A6801329A605B689A4236
S315080047C80ED9084A0846515802449160012006E065
S315080047D84FF4F171044800F051F9DAE7002038BDC2
S315080047E80120FCE7A80500208856000808B50146F8
S315080047F8024B1878FFF7C8FF08BD00BF200600203F
S3150800480810B50446012804D940F20221044800F0EC
S3150800481835F904EB4404E200024B1344587C10BDF6
S3150800482888560008A805002038B5FFF743FF1A4C34
S315080048384021601CFFF756FF2070184D4021681C60
S31508004848FFF750FF28702378FF2B1BD0FF2819D0B5
S31508004858134C002213492046FEF726FE1249204625
S31508004868FEF75BFE0120FBF7F0FC2046FEF769FE23
S31508004878D4F8C402FDF772FA00F02CF9B0F5FA6F0D
S3150800488805D338BD8521094800F0F8F8E0E74FF464
S31508004898FA6000F019F9F4E7DC0500202006002084
S315080048A864060020740000201000002088560008BE
S315080048B810B5064CD4F8C402FDF762FA2046FEF78E
S315080048C80FFE0020FBF7C1FC10BD00BF64060020E0
S315080048D870B506460D463F2906D82846FFF74AFF0B
S315080048E8012806D100240BE0B9210D4800F0C6F8C6
S315080048F8F3E7BD210A4800F0C1F8F3E70134A4B28A
S31508004908ABB2A3420BD900F0C3F9305DFFF732FF0B
S315080049180128F3D0C621024800F0B0F8EEE770BDCA
S315080049288856000870B506460D461F4BD3F8C402CC
S31508004938FCF7A0FF1D4B1C789CB91D48FFF756FFCE
S31508004948012801D0204670BD194B1B78013BDBB204
S315080049583E2BF7D8154B01221A70164B00221A70EF
S31508004968F0E7144B1B78013311481844FFF73EFF4C
S315080049780446012801D00024E4E70E4B1A780132D0
S31508004988D2B21A700A4B1B789A4201D00024D9E78A
S3150800499809493046FFF7AEFB044B00221A70054B4F
S315080049A81B782B70CEE700BF640600207409002028
S315080049B834090020750900203509002030B583B070
S315080049C8144B1878FFF71CFF08B30546402800D98A
S315080049D84025002405E09DF807200F4B1A55013499
S315080049E8E4B2A5420DD90DF107010A4B1878FFF76D
S315080049F8CBFE0128EFD04FF4A371084800F03EF823
S31508004A08E9E72B46044A8121054800F072FD03B000
S31508004A1830BD00BFDC050020680500208856000860
S31508004A286406002070B5044600F0A8FB0646214631
S31508004A380F4800F00CFD85B2002401E00134A4B249
S31508004A48AC420CD2315D0B4B1878FFF763FE012890
S31508004A58F4D04FF4B471084800F010F8EEE700F007
S31508004A688DFB402302460121014800F04AFD70BD2E
S31508004A7864060020200600208856000808B500F0BD
S31508004A8807F9FCE708B500F0F7F8012803D00B4B3F
S31508004A981B78012B00D008BDFFF700FE084B1B68E2
S31508004AA8084A1268134403F5FA739842F3D3034B7A
S31508004AB800221A70FFF7FEFAEDE700BF7C0900200E
S31508004AC87809002080090020014B1860704700BF4C
S31508004AD878090020014B1868704700BF780900203C
S31508004AE808B5054B1B78012B00D008BDFFF7D6FD86
S31508004AF8024B1860F9E700BF7C09002080090020EE
S31508004B0808B5044B01221A70FFF7EAFFFFF7BAFF48
S31508004B1808BD00BF7C09002008B5FFF7C7FA00F0F2
S31508004B28B3F8FFF799FDFFF7BBFC00F00DF8FFF7A0
S31508004B38E7FF08BD08B500F0ABF8FFF7A1FD00F0E0
S31508004B4817F8FFF79FFF08BD10B500F00FFAFFF733
S31508004B5813FA064C01232370FFF7E6FC002323709B
S31508004B68FFF762FE0223237010BD00BF0C00002069
S31508004B7800B583B00DF107011848FFF779FA01283F
S31508004B8810D00DF107011548FFF708FD012812D0C6
S31508004B980DF107011148FFF7C5FE012814D003B027
S31508004BA85DF804FB0E4B01221A709DF807100B4896
S31508004BB800F0FCF9E5E70A4B00221A709DF8071081
S31508004BC8064800F0F3F9E3E7054B02221A709DF848
S31508004BD80710024800F0EAF9E1E700BF8409002057
S31508004BE80C00002008B5FFF763FE08BD38B5044673
S31508004BF80D460E4B1B78012B09D00C4B1B7853B16D
S31508004C080A4B1B78022B0BD000F0C8F938BDC9B27D
S31508004C18FFF708FAF1E7E9B22046FFF7A3FCEFE742
S31508004C28E9B22046FFF754FEEEE700BF0C00002065
S31508004C38074B1B78022B05D0032B05D0012B05D073
S31508004C48402070473F20704700207047082070476B
S31508004C580C000020074B1B78022B05D0032B05D028
S31508004C68012B05D0402070473F2070470020704729
S31508004C78082070470C00002008B500F085F903469F
S31508004C8800B10123184608BD08B5FBF7D5FA08BDD3
S31508004C9808B5FBF7D6FA08BD014B00225A707047CB
S31508004CA8C4090020034BFE22DA7018710222A3F801
S31508004CB844207047C409002010B5054C002323700A
S31508004CC8FFF7EAFFFF23E3700123A4F8443010BD79
S31508004CD8C4090020064BFF22DA7000221A71597897
S31508004CE859719A71DA711A720622A3F84420704724
S31508004CF8C409002008B50020FFF7D4FF08BD000046
S31508004D08074BFF22DA70074A9A6400221A715A7109
S31508004D189A710722C3F807200822A3F84420704787
S31508004D28C4090020C4560008044BFF22DA704268FA
S31508004D389A640122A3F84420704700BFC4090020DA
S31508004D4808B53120FFF7AEFF08BD000038B5084C96
S31508004D58FF23E370002525716571FFF769FFA071C8
S31508004D68E571257265720723A4F8443038BD00BF7B
S31508004D78C409002038B5FFF78FFF0E4C01252570AA
S31508004D88FF23E3701023237100236371FFF750FF95
S31508004D98A071FFF75FFFE071FFF75CFFC0F307201C
S31508004DA820726572A5720823A4F84430FFF778FBC9
S31508004DB838BD00BFC409002038B505464478FFF752
S31508004DC837FF0138844210DC0A4C6A78A16C201D2A
S31508004DD8FFF790F9FF23E3706A78A36C1344A3647A
S31508004DE86B780133A4F8443038BD2220FFF75AFF00
S31508004DF8FAE700BFC409002038B504464578FFF726
S31508004E0817FF0138854211DC61680A4DA964627882
S31508004E18281DFFF76FF9FF23EB706278AB6C134414
S31508004E28AB6463780133A5F8443038BD2220FFF710
S31508004E3839FFFAE7C4090020F8B5054617460024DD
S31508004E4806E015F8013B1C44E4B2FFF721FF31469A
S31508004E584E1E0029F5D13C600120F8BD10B5084C56
S31508004E68FF23E370E21D4168A06CFFF7E5FF207198
S31508004E7800236371A3710823A4F8443010BD00BF4A
S31508004E88C409002038B505460D4B9C6CFFF7D0FEC3
S31508004E986A1C411E2046FFF707FB60B1084CFF2332
S31508004EA8E370FFF7C5FE0138A36C0344A364012326
S31508004EB8A4F8443038BD3120FFF7F4FEFAE700BFFE
S31508004EC8C409002038B504464578FFF7B1FE02380C
S31508004ED885420EDC114BFF22DA700122A3F8442022
S31508004EE8617851B9FFF7F0FA30B93120FFF7DAFEE1
S31508004EF802E02220FFF7D6FE38BDA21C074B986CA5
S31508004F08FFF7D2FA28B16178044A936C0B44936484
S31508004F18F2E73120FFF7C6FEEEE700BFC409002016
S31508004F2808B54168074B986CFFF7C2FA30B1054BCC
S31508004F38FF22DA700122A3F8442008BD3120FFF7C2
S31508004F48B1FEFAE7C409002008B5FFF7B3F8034B22
S31508004F58FF22DA700122A3F8442008BDC4090020FC
S31508004F6808B589B2FFF742FE08BD0000054B0022C6
S31508004F781A709A6483F84320A3F844209A705A70E2
S31508004F88704700BFC4090020034B1B780BB10120EA
S31508004F9870470020704700BFC4090020024B002252
S31508004FA883F84320704700BFC409002008B5037872
S31508004FB8FF2B04D0354A1278012A14D008BDFFF70A
S31508004FC8D9FE324B93F84330012B5AD02F4BB3F9FD
S31508004FD844100029F2DD1846012380F843300330CF
S31508004FE8FFF7BEFFEAE7C93B352B46D8DFE803F0EB
S31508004FF83345454245453F363C394545454545458A
S31508005008454545454545454545454545454545453A
S3150800501845454545454545454545241E1B214545C0
S315080050284527452A2D30FFF7C7FECAE7FFF7E4FEEE
S31508005038C7E7FFF779FEC4E7FFF710FFC1E7FFF7F1
S315080050485FFEBEE7FFF756FEBBE7FFF743FEB8E786
S31508005058FFF732FEB5E7FFF715FFB2E7FFF732FFAE
S31508005068AFE7FFF773FEACE7FFF75AFFA9E7FFF7C5
S315080050786BFFA6E7FFF764FEA3E72020FFF712FEFB
S315080050889FE71020FFF70EFEA0E700BFC40900201F
S315080050982023038000487047480000200A2303801D
S315080050A8004870476800002008B590F89C32032B22
S315080050B801D0002008BDFFF781FCFAE708B5FFF71D
S315080050C87DFC002008BD08B50846FFF7ABFC0020A4
S315080050D808BD000008B50B7813F0600F06D14B78A9
S315080050E80A2B14D00B2B17D0062B01D0002008BD8D
S315080050F84B881B0A212B04D00B491722FEF7C8FE3A
S31508005108F4E7CA88172A28BF17220849F6E70122AA
S315080051180749FEF7BDFEE9E78B7813B9044A136019
S31508005128E4E7FEF76BFBE1E7510000205A00002090
S31508005138100A002010B50446812100F0BAF90121A9
S31508005148204600F0B6F9002010BD000010B5044648
S3150800515840230222812100F0A1F9402302220121DD
S31508005168204600F09BF94023034A0121204600F017
S31508005178C8F9002010BD00BF600E0020004870471F
S31508005188600E002012230B8000487047900000200C
S3150800519804230B8000487047A4000020002393428C
S315080051A816D230B40BE0373401F8134000015C001E
S315080051B8013400250D550133DBB2934206D2040F9C
S315080051C8092CF0D8303401F81340EFE730BC7047A3
S315080051D87047000038B50A4B186804331C6804334E
S315080051E81B68C01800D138BD064D0822A91CFFF750
S315080051F8D5FF042205F112012046FFF7CFFFF2E793
S3150800520820F4F01FA800002008B51A230B80FFF722
S31508005218E1FF014808BD00BFA800002008B50A46F6
S3150800522828B105490548FEF717FE034808BD02498F
S315080052380248FEF711FEF8E7A00E0020FC56000803
S3150800524810B5044C0A4621460348FEF705FE2046D3
S3150800525810BD00BFA00E0020EC56000808B50A4687
S3150800526828B105490548FEF7F7FD034808BD024970
S315080052780248FEF7F1FDF8E7A00E0020CC56000814
S3150800528808B50A4628B105490548FEF7E5FD034865
S3150800529808BD02490248FEF7DFFDF8E7A00E002020
S315080052A8D456000808B500F57171D0F80004FEF761
S315080052B85DF908BD08B5C1EBC10293000344D3F8EC
S315080052C80822D0F80004FEF77DF908BD08B5C1EB39
S315080052D8C102930003449A6CD0F80004FEF7ABF9B0
S315080052E808BD08B5D0F80004FEF740FA08BD000066
S315080052F810B50446C3683BB1022B0FD09121084864
S31508005308FFF7BCFB012100E00021D4F80004FEF7F2
S3150800531816FAD4F80004FEF7E9F910BD0121F4E7F6
S315080053281057000810B50446D0F80004FEF70AFA24
S315080053382268D2F8003E43F00103C2F8003E236A09
S3150800534823B1044A136943F006031361FAF77EFF8B
S3150800535810BD00BF00ED00E010B50446FAF777FF68
S31508005368D4F80004FEF7F7F910BD08B5D0F800041C
S31508005378FEF70CFA08BD08B5D0F80004FEF704FADB
S3150800538808BD10B504460120FAF75FFFD4F80004F3
S31508005398FEF7FEF910BD10B504460020FAF755FFCA
S315080053A8D4F80004FEF7F6F910BD000003780BB12F
S315080053B80020704710B503461748C0F80034C3F8EC
S315080053C8C4024FF0A0430360062343600222C2606A
S315080053D80023036182610122C26103624362C362D8
S315080053E80363FCF7C1F880B90B4C80212046FCF70B
S315080053F862FE402200212046FCF739FE8022012160
S315080054082046FCF734FE002010BD40F2251103485B
S31508005418FFF734FBE8E700BF140A00201057000816
S31508005428D0F8C43211F0800F08D101F07F01C1EB22
S31508005438C1018A00134493F8FE01704701F07F0101
S31508005448C1EBC1018A00134493F83E00704708B5BA
S31508005458D0F8C402FCF760FD08BD18B1022803D0CD
S3150800546803207047002070470120704708B5D0F818
S31508005478C402FCF746F9FFF7F0FF08BD08B5D0F8EF
S31508005488C402FCF709F9FFF7E8FF08BD08B5D0F824
S31508005498C402FCF716F9FFF7E0FF08BD10B51C466D
S315080054A813462246D0F8C402FCF790FCFFF7D5FF4E
S315080054B810BD08B5D0F8C402FCF7C9FCFFF7CDFF44
S315080054C808BD08B5D0F8C402FCF759FDFFF7C5FFB3
S315080054D808BD08B5D0F8C402FCF792FDFFF7BDFF72
S315080054E808BD08B5D0F8C402FCF75CFCFFF7B5FFA1
S315080054F808BD08B5D0F8C402FCF717FDFFF7ADFFDD
S3150800550808BD08B5D0F8C402FCF7D8FCFFF7A5FF14
S3150800551808BD000070B50D4E0D4CA41BA41000253F
S31508005528A54209D10B4E0C4C00F018F8A41BA41080
S315080055380025A54205D170BD56F82530984701358E
S31508005548EEE756F8253098470135F2E7345700084C
S31508005558345700083457000838570008F8B500BF0C
S31508005568F8BC08BC9E467047F8B500BFF8BC08BC2E
S309080055789E46704786
S3150800557C00000000000000000102030406070809E9
S3150800558C0000000001020304433A2F576F726B2F79
S3150800559C736F6674776172652F4F70656E424C54E3
S315080055AC2F5461726765742F536F757263652F413B
S315080055BC524D434D375F53544D333246372F636143
S315080055CC6E2E630005020602060307030803090389
S315080055DC09040A040B040C040C050D050E050F052D
S315080055EC0F0610061007100800800008008000003F
S315080055FC0100000000000108008000000200000005
S3150800560C008001080080000003000000000002086A
S3150800561C000002000400000000000408000004005A
S3150800562C0500000000000808000004000600000041
S3150800563C00000C080000040007000000433A2F572E
S3150800564C6F726B2F736F6674776172652F4F706507
S3150800565C6E424C542F5461726765742F536F757272
S3150800566C63652F41524D434D375F53544D33324684
S3150800567C372F72733233322E63000000433A2F579A
S3150800568C6F726B2F736F6674776172652F4F7065C7
S3150800569C6E424C542F5461726765742F536F757232
S315080056AC63652F41524D434D375F53544D33324644
S315080056BC372F7573622E63004F70656E424C54001B
S315080056CC44656661756C740057696E555342204281
S315080056DC756C6B20496E74657266616365000000B3
S315080056EC4F70656E424C542055736572000000006D
S315080056FC57696E5553422042756C6B204465766922
S3150800570C636500002E2E2F5553425F444556494378
S3150800571C452F5461726765742F757362645F636F86
S30D0800572C6E662E630000000002
S30908005734ED0100086D
S30908005738C90100088D
S3150800573C0024F40001000000100000000400000022
S3150800574C555100083D510008DD50000800000000C6
S3150800575C00000000C5500008CF500008B1500008E2
S3150800576C000000000000000000000000995000082E
S3150800577C00000000A550000809022000010100C025
S3150800578C320904000002FF000000070581024000F0
S3150800579CFF070501024000FF0A0600020000004050
S315080057AC010000008D510008995100084952000863
S315080057BC2552000811520008655200088952000843
S315080057CC1201000200000040501DAC6000020102EC
S315080057DC03010000040309041A030000000000007A
S315080057EC000000000000000000000000000000009F
S309080057FC000000009B
S70508000735B6
